:100000008128FF3FFF3FFF3FFF00030E8301A40055
:100010000408A3000A08A5008A017008A6000C10B5
:100020008F018E012008210203186428392801302D
:100030008700A20A3030A100612802308700A20A9E
:100040003030A100612804308700A20A3030A100BE
:10005000612807308700A20A3030A100612887019B
:10006000A20A0830A10061288701A2010830A1007E
:1000700061282208003A031917282208033A0319B5
:1000800017282208013A03191D282208043A0319E7
:100090001D282208023A031923282208053A0319C9
:1000A00023282208063A031929282208083A0319A6
:1000B00029282208073A03192F282208093A031988
:1000C00034280130A0006528A00A2608F000250881
:1000D0008A0023088400240E8300FF0E7F0E09008F
:1000E000C0308B000313831687010C1480308312F9
:1000F0008F008E0101309000A2010130A000A1010B
:10010000080070208228FF3FFF3FFF3FFF3FFF3F77
:02400E00EA3F87
:00000001FF
